:020000040000FA
:0200000015D019
:08000800006ED8CF02F0E0CF3A
:1000100001F0F2B2B6EC00F09EB037EC00F000D088
:1000200001C0E0FF005002C0D8FF1000806A816A62
:10003000826A0F0EC16E070EB46EF26A90EC00F089
:10004000ADEC00F0356A82EC00F0D09EF28EF28CBE
:1000500005EC01F00000000000000000000035A0E9
:10006000F9D7359041EC00F000000000F3D7CD90B7
:100070003450CF6E3350CE6E35809E909D80CD80B3
:100080001200100E0E5CD8A00AD010EE12F020EE76
:1000900022F00E6A32D81FD82AD80CD809D00E50B8
:1000A0000F6E2BD818D823D81CD80F2EFDD702D806
:1000B0000E2A1200FC0E8016030E8116E6CF10F0F9
:1000C000104610461050FC0B81121050030B80128A
:1000D000DECF82FF1200030E8116FC0E8016826AAC
:1000E00012008096000080840000809412008086B8
:1000F00000008084000080941200809A00000000BC
:10010000808A1200E00E346E000E336E840ECD6EC7
:1001100034C0CFFF33C0CEFF9E909D80CD801200B3
:10012000929A92969294809A8096809410EE12F011
:10013000200E0F6EE6680F2EFDD792909292939448
:1001400093969398939A939C939E000E946E808AB4
:100150000E6A010E326E116E120093809382F18C42
:10016000F292F288056A080E066E1200BBEC00F0EF
:10017000F292F2881200D89081B2D8800A320550EB
:10018000046ED8900436010ED8B0E828FA6E980EA6
:100190000424D8B0FA2AF96E02D00AD016D0062E5E
:1001A0001200010E056E060E066E0A50076E120052
:1001B000062E1200020E056E080E066E0A50086E1C
:1001C000D8900832D89008321200062E1200000E85
:1001D000056E080E066E300E076212000A50096E98
:1001E00000EE12F0085009C0EBFF12000A0E0B6E71
:1001F000010E0D6EC80E0C6E000000000C2EFCD718
:100200000D2EF8D70B2EF4D712000A0E0B6EFA0E35
:100210000D6EC80E0C6E000000000C2EFCD70D2ECB
:10022000F8D70B2EF4D712000A0E0B6E0D6EC80E07
:100230000C6E000000000C2EFCD70D2EF8D70B2EF4
:10024000F5D712000A0E0B6E010E0D6E320E0C6EFB
:10025000000000000C2EFCD70D2EF8D70B2EF4D783
:10026000120005EC01F005EC01F005EC01F005ECE5
:0402700001F0120087
:020000040030CA
:0E000000FF36FEFEFFFDFAFFFFFFFFFFFFFFD2
:00000001FF
